:10000000F3EF04F00000000000EF00F0000000003B
:0A0010000000000000000000F3D71C
:10001C0035CA04F08B92026A036A800E0318006ED4
:10002C00800E005C02E1080E025C1FE2800E0414DC
:10003C00016E0150800A02E18B8201D08B921A0E64
:10004C000D6E0D2EFED70000043604908B842A0E04
:10005C000D6E0D2EFED700008B941A0E0D6E0D2E0C
:0C006C00FED70000024A032AD8D7120079
:100078008B904F0E0D6E0D2EFED7000000002CCA7F
:1000880035FAC8DF34CA35FAC5DF2CCA35FAC2DFFB
:1000980033CA35FABFDF2CCA35FABCDF32CA35FAA3
:1000A800B9DF2CCA35FAB6DF31CA35FAB3DF2CCA44
:1000B80035FAB0DF30CA35FAADDF2CCA35FAAADF17
:1000C8002FCA35FAA7DF2CCA35FAA4DF2ECA35FAAB
:1000D800A1DF2CCA35FA9EDF2DCA35FA9BDF350E13
:1000E8000D6E0D2EFED78B801A0E0D6E0D2EFED7BF
:0400F80000001200F2
:1000FC000A012A6B2B6B800E2B19006E800E005C94
:10010C0002E1080E2A5D15E22A51010F2C6F2D6BAE
:10011C002E6B2F6B306B316B326B336B346BA6DF0A
:10012C006A0E0D6E0D2EFED700000A012A4B2B2BEA
:04013C00E2D71200F4
:0E014000ACB202D00000FCD72ACAADFF1200FC
:10014E00086A096A100E0C6E01340836093604501E
:10015E00085E0550D8A0053C095ED8B007D0045003
:10016E0008260550D8B0053C0926D8900036013631
:06017E000C2EEAD712006E
:1001840022CA02F023CA03F002C000F003C001F047
:10019400024A032A00C0E9FF01C0EAFFEE5201E06F
:1001A400F3D70A012251025C006E23510358016EF9
:0A01B400010E005E000E015A120059
:1001BE000A01266B276B22CAE9FF23CAEAFFEE501B
:1001CE000008D8B0B2D022CAE9FF23CAEAFFEECFA8
:1001DE0001F0030E006E01C028FA000E296F0050C8
:1001EE0005E0283728912937FF0FFAD7246B256BA6
:1001FE00800E2519006E800E005C02E1080E245D53
:10020E00D8B08CD024512625006E25512721016EA1
:10021E00080E0024E16E090E0120E26E24512825FD
:10022E00006E25512921016E7F0E0024E96E000E0D
:10023E000120EA6EEECFE6FF2451010F2C6F080E5F
:10024E002425E96E090E2521EA6EEECF2DFA080E51
:10025E002425006E000E2521016E080E0024E96E85
:10026E00090E0120EA6EEECF2EFA100E2425006E36
:10027E00000E2521016E080E0024E96E090E0120E4
:10028E00EA6EEECF2FFA180E2425006E000E2521F1
:10029E00016E080E0024E96E090E0120EA6EEECF03
:1002AE0030FA200E2425006E000E2521016E080E58
:1002BE000024E96E090E0120EA6EEECF31FA280E07
:1002CE002425006E000E2521016E080E0024E96E15
:1002DE00090E0120EA6EEECF32FA300E2425006EA2
:1002EE00000E2521016E080E0024E96E090E012074
:1002FE00EA6EEECF33FA380E2425006E000E25215D
:10030E00016E080E0024E96E090E0120EA6EEECF92
:10031E0034FAABDE0A01244B252B6AD7080E2627AA
:0C032E00000E2723224B232B46D7120081
:10033A0024CAF6FF25CAF7FF26CAF8FF0900F5CF37
:10034A0000F0005218E024CAF6FF25CAF7FF26CAB1
:10035A00F8FF0900F5CF00F022CAE1FF23CAE2FF45
:10036A0000C0E6FF0A01224B232B010E2427000EB0
:10037A0025232623DDD722CAE1FF23CAE2FFE66A44
:02038A0012005F
:10038C000A01266B050E265D0AE226512425E16E34
:10039C00000E2521E26E200EE66E262BF3D7265199
:1003AC002425E16E000E2521E26EE66A2607265111
:1003BC002425276F000E2521286F0A0E046E000ECF
:1003CC00056E22CA00F023CA01F0BBDE08C000F0A3
:1003DC0009C001F0300E002627CAE1FF28CAE2FF4F
:1003EC0000C0E6FF0A0E046E000E056E22CA00F075
:1003FC0023CA01F0A6DE00C022FA01C023FA000EC7
:10040C00011802E1000E001801E102D02607CFD737
:02041C001200CC
:10041E000A01256B22CAE9FF23CAEAFFEECF24FAAE
:10042E002451000A0EE024CA2AFA83DE0A01252B83
:10043E0025512225E96E000E2321EA6EEECF24FA15
:04044E00EFD71200D2
:1004520022CA04F023CA05F004C0E9FF05C0EAFF7E
:10046200EE5203E0044A052AF7D704C002F005C0A1
:1004720003F0044A052A24CA00F025CA01F00A0141
:10048200244B252B00C0E9FF01C0EAFF02C0E1FFB7
:1004920003C0E2FFEECFE6FF02C0E9FF03C0EAFFBE
:1004A200EE5201E0E2D722CA00F023CA01F01200A4
:1004B2000A01226B236B160E246F000E256F226B2E
:1004C200236B800E2319006E800E005C02E1080E81
:1004D200225D72E22251010F2C6F22512425E96E16
:1004E20023512521EA6EEECF2DFA080E2425006E47
:1004F200000E2521016E22510024E96E23510120B4
:10050200EA6EEECF2EFA100E2425006E000E252183
:10051200016E22510024E96E23510120EA6EEECFD2
:100522002FFA180E2425006E000E2521016E22518D
:100532000024E96E23510120EA6EEECF30FA200E3C
:100542002425006E000E2521016E22510024E96E41
:1005520023510120EA6EEECF31FA280E2425006ED7
:10056200000E2521016E22510024E96E2351012043
:10057200EA6EEECF32FA300E2425006E000E2521EF
:10058200016E22510024E96E23510120EA6EEECF62
:1005920033FA380E2425006E000E2521016E2251F9
:1005A2000024E96E23510120EA6EEECF34FA63DDB6
:0A05B2000A01224B232B85D712000B
:1005BC000D0E0A012A6FBEDD0A0E0A012A6FBADD82
:0205CC0012001B
:1005CE000B6A0A6A096A00500402F4CF09F0F3CFED
:1005DE0008F001500502F4CF0BF0F3CF0AF00050F3
:1005EE000502F3500926F4500A22E86A0B22015044
:1005FE000402F3500926F4500A22E86A0B2208C0BE
:10060E0000F009C001F00AC002F00BC003F01200A6
:10061E00400E0901946F010E956F2A0E966F0A0E09
:10062E00976FFF0E8C6FFF0E8D6F000E8E6F000E8C
:10063E008F6FFF0E986FFF0E996F000E9A6F000E60
:10064E009B6FFF0E906FFF0E916F000E926F000E5C
:10065E00936FAC8A900EAB6E948E949C9EAA03D030
:08066E00AECF00F0FBD7120033
:100676000900F5CFE6FF0006FBE10106F9E11200ED
:10068600826A0F013A6B948E949C949094948B9406
:1006960094928B823F0E806E386B2F0E926E546B47
:0E06A600FF0E816E830E936E396B606A120038
:1006B400090E0B6E1E0E0C6EE40E0D6E0D2EFED783
:1006C4000C2EFCD70B2EFAD700000F0E0A012C6F4C
:1006D4002D6B2E6B2F6B306B316B326B336B346B3A
:1006E400C9DC090E0A012C6F2D6B2E6B2F6B306B3E
:1006F400316B326B336B346BBDDC0A0E0A012C6F29
:100704002D6B2E6B2F6B306B316B326B336B346B09
:10071400B1DC0B0E0A012C6F070E2D6F070E2E6F26
:10072400070E2F6F070E306F070E316F070E326FF3
:10073400070E336F070E346F9DDC0C0E0A012C6F0D
:10074400010E2D6F010E2E6F010E2F6F010E306FF3
:10075400010E316F010E326F010E336F010E346FD3
:1007640089DC2A0E0C6E8D0E0D6E0D2EFED70C2E0E
:10077400FCD700000000C0DCD00E0C6EC90E0D6E5C
:0E0784000D2EFED70C2EFCD700000000120038
:100792000000D89058A003D0D89016BED8804E360C
:1007A20046363E3636362E3626361E361636D89023
:1007B20058A003D0D89017BED8804F3647363F3660
:1007C20037362F3627361F361736D89058A003D023
:1007D200D89018BED8805036483640363836303633
:1007E200283620361836D89058A003D0D89019BE93
:1007F200D880513649364136393631362936213696
:100802001936D89058A003D0D8901ABED880523644
:100812004A3642363A3632362A3622361A36D89096
:1008220058A003D0D8901BBED88053364B364336DF
:100832003B3633362B3623361B36D89058A003D09E
:10084200D8901CBED88054364C3644363C363436AA
:100852002C3624361C36D89058A003D0D8901DBE12
:10086200D88055364D3645363D3635362D36253609
:100872001D360000150E0C6EC60E0D6E0D2EFED727
:080882000C2EFCD7000012004F
:10088A00080E0A01256F010E246F800E000A006E01
:10089A00800E2519005C23E224512215016E0150B5
:1008AA0000080CE22351010A04E12A0E2A6F43DCF4
:1008BA0004D0310E0A012A6F3EDC0CD00A01235102
:1008CA00010A04E12E0E2A6F36DC04D0300E0A012A
:1008DA002A6F31DC0A01243724912507D6D7120062
:1008EA0022CAF6FF23CAF7FF24CAF8FF0900F5CF88
:1008FA0000F0005211E022CAF6FF23CAF7FF24CA09
:10090A00F8FF0900F5CF2AFA16DC010E0A012227A0
:10091A00000E23232423E4D71A0E0D6E0D2EFED7C4
:04092A0000001200B7
:10092E00160E0901886F000E896F056A066A036A42
:10093E00046A056A066A000E065C02E1080E055C92
:10094E004AE205500A012225E96E06502321EA6E7D
:10095E00EECF01F0030E006E01C007F0000E086E20
:10096E00005005E0073607900836FF0FFAD7036AE6
:10097E00046A000E045C02E1080E035C29E20350D7
:10098E000724006E04500820016E7F0E0024E96ECD
:10099E00000E0120EA6E05C000F006C001F0003620
:1009AE000090013600360090013600360090013678
:1009BE000350002604500122005009018825E16EE3
:1009CE0001508921E26EEECFE6FF034A042AD1D709
:0809DE00054A062AB0D71200F9
:1009E60088EC0DF09B6A700ED36E9B8CD26A010E5A
:1009F600566E000E576E0901066B076B800E0719BF
:100A0600006E800E005C02E1800E065D0AE2080EB2
:100A16000625E16E090E0721E26EE66A064B072BF4
:100A2600EDD72EDE8B80160E0901886F000E896FBA
:100A3600066B076B800E0719006E800E005C02E1E4
:100A4600100E065D0AE2160E0625E16E000E07215F
:100A5600E26EE66A064B072BEDD7010E156EB886D9
:100A6600030EB06E400EAF6EAC84D6DD090E0B6E73
:100A76001E0E0C6EE40E0D6E0D2EFED70C2EFCD740
:100A86000B2EFAD7000097DDE10E0A01226F1A0E2F
:100A9600236F000E246F26DF0901066B076B800E9D
:100AA6000719006E800E005C02E1090E065D1AE26F
:100AB600030E006E000E016E06C904F007C905F0AC
:100AC60083DD590E0024E96E000E0120EA6EEECF9A
:100AD60022FAEECF23FAEECF24FA04DF0901064B01
:100AE600072BDDD7520E0B6E2B0E0C6E000E0D6E05
:100AF6000D2EFED70C2EFCD70B2EFAD700005BDD91
:100B0600FD0E0A01226F1A0E236F000E246FEADE15
:100B160051D00D2EFED70C2EFCD70B2EFAD7000087
:100B26004ADD5E0E0A01226F190E236F000E246F36
:100B3600D9DE0901066B076B800E0719006E800E61
:100B4600005C02E1080E065D27E2280E0625006E0F
:100B5600020E0721016E00C004F901C005F97F0EDF
:100B66000024E96E000E0120EA6EEECF00F000C010
:100B760083F8770E0625E16E000E0721E26E00C0AF
:100B8600E6FF83C822FA010E0A01236F7BDE13DD1E
:100B96000901064B072BD0D7520E0B6E2B0E0C6E8F
:100BA600000E0D6E0D2EFED70C2EFCD70B2EFAD78F
:100BB600000001DD010E586E7ADD7EEC00F0F29E3B
:100BC60009018A6B8B6B010E586E2E0E0A01226F7D
:100BD6001A0E236F000E246F85DE9E0E0A01226F09
:100BE600090E236FF40E246F1A0E256F000E266F62
:100BF6009DEC01F04E0E0A01226F1A0E236F000EB5
:100C0600246F70DE9E0E0A01226F090E236FDFEC41
:100C160000F0A30E0B6E570E0C6E020E0D6E0D2E0F
:100C2600FED70C2EFCD70B2EFAD70000C4DC840EA0
:100C36000801816F080E826F0901066B076B800E33
:100C46000719006E800E005C02E1480E065D0AE29E
:100C5600840E0625E16E080E0721E26EE66A064B53
:100C6600072BEDD7840E0801816F080E826F81C8AD
:100C760022FA82C823FA910E0A01246F190E256FF3
:100C8600000E266F9DEC01F081C822FA82C823FA75
:100C9600C2EC00F0800E0118026E800E025C02E1CA
:100CA600400E005C0BE281C822FA82C823FA7F0E4E
:100CB600246F080E256F29EC02F0E6D70801C46BF5
:100CC60081C820FA82C821FA6C0E0A01226F1A0E18
:100CD600236F000E246F06DE20CA22FA21CA23FAE9
:100CE6000FEC02F068DC81C822FA82C823FAC2EC53
:100CF60000F000C004F901C005F900C022FA01C0E5
:100D060023FA9E0E246F090E256FC6EC01F0CD0E58
:100D1600226F1A0E236F000E246FE4DD9E0E0A0169
:100D2600226F090E236F0FEC02F045DC20CA22FA6F
:100D360021CA23FAF9DD59EC02F0586A1E6B1F6BC3
:100D460081C820FA82C821FAA00E226F1A0E236FDC
:100D5600000E246FC7DD010E09018A6F000E8B6F2E
:100D6600586A800E006E800E8B19005C02E18A5173
:100D76000708D8B017D18A6B8B6BBDD00A011E51FC
:100D8600400809019C6F1FCA9DF9000E9D57066B0E
:100D9600076B800E0719006E800E9D19005C02E13C
:100DA6009C51065D1BE2080E0625E16E090E072121
:100DB600E26E06510A012025006E090107510A015B
:100DC6002121016E1E510024E96E1F510120EA6E99
:100DD600EECFE6FF0901064B072BDBD70A011E51B2
:100DE6004008006E1FCA01F0000E015600500808A8
:100DF600026E01C003F0000E035602C09CF903C048
:100E06009DF9800E006E800E0318005C02E1025010
:100E1600000832E2800E09019D19006E800E005C0A
:100E260002E1080E9C5D28E29CC906F99DC907F9F6
:100E3600800E0719006E800E005C02E1080E065D4A
:100E46001BE2080E0625E16E090E0721E26E065129
:100E56000A012025006E090107510A012121016EB0
:100E66001E510024E96E1F510120EA6EEECFE6FF07
:100E76000901064B072BDCD70901106B76D01ECA79
:100E860022FA1FCA23FA9E0E0A01246F090E256F45
:100E9600C6EC01F09E0E226F090E236F0FEC02F0D6
:100EA6003E0E2A6FA0EC00F00901066B076B800E60
:100EB6000719006E800E005C02E1080E065D19E25D
:100EC600080E0625E16E090E0721E26E0A011E5183
:100ED6002025006E1F512121016E090106510024B3
:100EE600E96E07510120EA6EEECFE6FF064B072BAF
:100EF600DED7106B3AD0000E0A011F1902E1380E38
:100F06001E19D8B43BD7000E1F1902E1390E1E195F
:100F1600D8B434D7000E1F1902E13A0E1E19D8B400
:100F26002DD7000E1F1902E13B0E1E19D8B426D785
:100F3600000E1F1902E13C0E1E19D8B41FD7000E71
:100F46001F1902E13D0E1E19D8B418D7000E1F193D
:100F560002E13E0E1E19D8B411D7000E1F1902E188
:100F66003F0E1E19D8B40AD78AD7680E0C6EE40E47
:100F76000D6E0A010D2EFDD70C2EFBD700001E4B61
:100F86001F2B800E006E800E1F19005C02E11E51A1
:100F96003F0802E21E6B1F6B080E226F090E236FBD
:100FA600C3DC02D059EC02F0586AC9EC03F0020E19
:100FB6000B6EA00E0C6E920E0D6E0D2EFED70C2E25
:100FC600FCD70B2EFAD7000009018A4B8B2BC8D60B
:020FD600FFD743
:101B100010EE59F0260E006E010E016EE80EF66E04
:101B2000190EF76E000EF86E3BEC03F010EE56F057
:101B3000020E006E010E016E0A0EF66E1B0EF76E9F
:101B4000000EF86E3BEC03F010EE15F0010E006E87
:101B5000010E016E0E0EF66E1B0EF76E000EF86E85
:101B60003BEC03F010EE7FF0020E006E090E016EEA
:101B7000D80EF66E0F0EF76E000EF86E3BEC03F00B
:021B8000120051
:100FD80000000000000000007E81A581BD99817E8F
:100FE8007EFFDBFFC3E7FF7E6CFEFEFE7C38100051
:100FF80010387CFE7C381000387C38FEFE7C387C4B
:101008001010387CFE7C387C0000183C3C1800002E
:10101800FFFFE7C3C3E7FFFF003C664242663C00B0
:10102800FFC399BDBD99C3FF0F070F7DCCCCCC780A
:101038003C6666663C187E183F333F303070F0E0FF
:101048007F637F636367E6C0995A3CE7E73C5A9938
:1010580080E0F8FEF8E08000020E3EFE3E0E020040
:10106800183C7E18187E3C18666666666600660040
:101078007FDBDB7B1B1B1B003E63386C6C38CC783A
:10108800000000007E7E7E00183C7E187E3C18FF23
:10109800183C7E1818181800181818187E3C1800E4
:1010A80000180CFE0C180000003060FE60300000D4
:1010B8000000C0C0C0FE0000002466FF66240000D7
:1010C80000183C7EFFFF000000FFFF7E3C18000078
:1010D8000000000000000000404040404000400088
:1010E80090900000000000005050F850F850500058
:1010F8002078A07028F02000C8C8102040989800D8
:10110800708850205488740060204000000000005F
:10111800204080808040200020100808081020000F
:101128000020A87070A8200000002020F8202000CF
:10113800000000000060204000000000F8000000EF
:1011480000000000006060000204081020408000D9
:10115800708898A8C888700040C040404040E000AF
:10116800708808102040F8007088081008887000FF
:1011780008182848FC080800F88080F008887000E3
:10118800204080F088887000F80810204040400017
:10119800708888708888700070888878080870005F
:1011A8000000606000606000000060600060602017
:1011B80010204080402010000000F800F8000000D7
:1011C800804020102040800078840408100010001F
:1011D800708888A8B880780020508888F8888800A7
:1011E800F08888F08888F000708880808088700097
:1011F800F08888888888F000F88080E08080F8008F
:10120800F88080E0808080007088808098887800EE
:10121800888888F888888800E04040404040E0009E
:1012280038101010109060008890A0C0A09088001E
:10123800808080808080F80082C6AA9282828200A4
:1012480084C4A4948C8484007088888888887000FA
:10125800F08888F08080800070888888A89068006E
:10126800F08888F0A09088007088807008887000E6
:10127800F82020202020200088888888888870000E
:1012880088888850502020008282828292926C0046
:10129800888850205088880088888850202020001E
:1012A800F80810204080F800E08080808080E0000E
:1012B8008040201008040200E02020202020E000C8
:1012C8002050880000000000000000000000F80026
:1012D80040200000000000000000700878887400BA
:1012E8008080B0C888C8B00000007088808870000E
:1012F800080868988898680000007088F88070006E
:10130800304840E040404000000034484838083049
:101318008080B0C888888800200060202020700065
:10132800100030101010906080808890A0D0880045
:10133800C04040404040E0000000EC929292920091
:101348000000B0C88888880000007088888870000D
:101358000000B0C8C8B08080000068989868080885
:101368000000B0C880808000000078807008F0001D
:101378004040E0404050200000008888889868007D
:1013880000008888885020000000828292926C00B9
:1013980000008850205088000000888898680870ED
:1013A8000000F8102040F8001020204020201000F5
:1013B8004040400040404000402020102020400095
:1013C80076DC0000000000000010386CC6C6FE0085
:1013D8003E60C0603E080418004800CCCCCCCC76F7
:1013E80018200078CCFCC078102800780C7CCC76CB
:1013F800004800780C7CCC76300800780C7CCC76E1
:10140800483000780C7CCC7678CCC0CC781008308A
:1014180030488478CCFCC07800480078CCFCC07890
:1014280030080078CCFCC0780048003030303030CC
:1014380030480030303030306010003030303030DC
:1014480048003078CCCCFCCC3048304884FC8484CC
:10145800182000F880F080F8000000661977887777
:101468000000000F143E448730488478CCCCCC78F8
:1014780000480078CCCCCC7860100078CCCCCC7804
:1014880030488400CCCCCC76601000CCCCCCCC7668
:101498004800CCCCCC7C0CF84400386CC6C66C3800
:1014A800240066666666663C00081C28281C08003E
:1014B8001C22207020225C0044281010381038109C
:1014C800F0888AF7828283000608083C10106000C2
:1014D800182000780C7CCC76182000303030303062
:1014E80018200078CCCCCC78182000CCCCCCCC768A
:1014F800807804F8CCCCCCCC807E01C6E6D6CEC6AB
:1015080000780C7CCC7600FE0078CCCCCC7800FC43
:10151800000018183060663CFF80808000000000E2
:10152800FF0101010000000040C44850264982071D
:1015380040C44850264A9F020030003030303030D6
:101548000012244890482412004824120912244802
:1015580049009200490092006D00B6006D00B60087
:10156800AA55AA55AA55AA551010101010101010F7
:1015780010101010F0101010101010F010F01010C3
:1015880028282828E828282800000000F8282828E3
:10159800000000F010F01010282828E808E8282893
:1015A8002828282828282828000000F808E82828BB
:1015B800282828E808F8000028282828F80000002B
:1015C800101010F010F0000000000000F0101010D3
:1015D800101010101F00000010101010FF00000065
:1015E80000000000FF101010101010101F10101035
:1015F80000000000FF00000010101010FF10101075
:101608001010101F101F1010282828283F282828DD
:101618002828282F203F00000000003F202F2828DE
:10162800282828EF00FF0000000000FF00EF28280E
:101638002828282F202F2828000000FF00FF00005E
:10164800282828EF00EF2828101010FF00FF0000BE
:1016580028282828FF000000000000FF00FF1010C5
:1016680000000000FF282828282828283F0000001C
:101678001010101F101F00000000001F101F101076
:10168800000000003F28282828282828FF28282884
:10169800101010FF10FF101010101010F0000000B4
:1016A800000000001F101010FFFFFFFFFFFFFFFFEB
:1016B80000000000FFFFFF00E0E0E0E0E0E0E0E025
:1016C8000707070707070707FFFFFFFF00000000DE
:1016D80000000002344C4C32005C22223C44447826
:1016E8007E424240404040400000027CA8282844F6
:1016F800007E6130180810200000087F88888870F4
:101708000000002244447A800000007C1010101071
:10171800001C083E4141413E00003844447C44449A
:101728003C66C3C3C36624660C10081C2222221C14
:10173800000000006C92926C00011A262A322C409C
:101748000018202030202018003C424242424242E9
:1017580000007E007E007E000008083E0808003E6B
:10176800001008040810003E000408100804003E99
:101778000006090908080800000008080848483059
:10178800000008003E0008000060920C60920C0007
:101798006090600000000000000000307830000019
:1017A800000000002000000000030404C828100006
:1017B8000000007C42424200182408103C0000004F
:1017C8000000003E3E3E3E00000000000000000019
:0217D8002000EF
:1017DA0020536F75726365203A20746573745F31A4
:1017EA00384632364B32325F646566696C656D65C0
:1017FA006E745F74657874655F646563616C616754
:10180A00655F3634626974735F61736D5F5F313926
:0A181A00313230322E63200D0A0037
:101824002050726F6A6574203A20746573745F3156
:10183400384632364B32325F646566696C656D6575
:101844006E745F74657874655F646563616C616709
:10185400655F3634626974735F61736D5F3139310A
:0A186400322E6D637070690D0A00EA
:10186E00204469726563746F7279203A20433A5C42
:10187E005F4D696B726F435C5F4D657350726F6A3B
:10188E006574735F4D696B726F435C5F4D61783742
:10189E003231395F345F365F385F4D617472696320
:0818AE0065387838200D0A00AE
:1018B6002032204D6F64756C6573204E657720521B
:1018C600657665727365203478204D61747269633C
:1018D6006573203878382061766563204D41583726
:0A18E60031323920434D530D0A0042
:1018F000205465726D696E616C20706F7572206422
:1019000069616C6F67756520657420566973752011
:10191000206465726F756C656D656E742070726F92
:091920006772616D6D650D0A002E
:1019290020205265766572736520486F72697A6FF7
:101939006E74616C206465732062697473206465D8
:10194900206C6120666F6E7465206C6574747265B5
:0519590020450D0A000D
:10195E00205265746F757220E02041666669636877
:10196E00616765204F726967696E616C20466F6EA4
:10197E007420387838203A206C657474726520456E
:03198E000D0A003F
:1019910020202020202020205061756C2057616E6E
:1019A1007420746F206B696C6C207468652062759B
:0D19B1006720303132333435363738390095
:1019BE0020416666696368616765204F7269676971
:1019CE006E616C20466F6E7420387838203A206C29
:0A19DE00657474726520450D0A005F
:1019E800861A006E1800241800DA1700B61800F0DE
:0E19F8001800B91A00021B00061B000C1B0091
:081A0600FE6268786862FE00D0
:101A0E002041666669636861676520524556455296
:101A1E0053454420206C657474726520450D0A0090
:101A2E002054657874652064652044657061727415
:101A3E00203A203C30313233343536373E0D0A00F1
:101A4E002041666669636865205445585445207583
:0E1A5E0072204D617472696365733E0D0A005B
:101A6C0020496E6974206D65737361676520363427
:0A1A7C0020636172733A0D0A200026
:101A8600204D696B726F6320372E362E3020313829
:0A1A96004632364B3232200D0A00B2
:101AA0002044656D6D617261676520646563616C7A
:091AB000616765203A200D0A006F
:101AB90020416C696D203D332C3320E020342C36D5
:041AC900560D0A00AC
:101ACD00204C6F6E67756572206D65737361676508
:041ADD00203D200088
:101AE1002050726573656E746174696F6E203A205F
:031AF1000D0A00DB
:091AF4003031323334353637004D
:051AFD00474F0D0A0037
:041B0200200D0A00A8
:041B0600200D0A00A4
:021B0A000100D8
:021B0C002000B7
:011B0E0001D5
:020000040030CA
:0D000100381F3CFFBF81FF0FC00FE00F4014
:00000001FF
